:020000040000FA
:02000000812855
:02000800722A5A
:10001000D10000300D28D1004030D20048207C3083
:10002000512052085120510851204D20182008001D
:100030000A30CC001B28CC0B1A28080028305E227E
:10004000383008203930082014300820703008205B
:10005000563008206C300820C8305E223830082026
:100060000C3008200130082001305E2251220800A7
:1000700044208A110A12D00A0319CF0A003E03193C
:1000800043280B20382808004F088A0050088200B7
:100090008514051405108510080085140510051435
:1000A0000800D3000830D4000510D31B05148514B4
:1000B0008510D30DD40B5428831605148312851490
:1000C0000000851083160510831208000830D40044
:1000D0008316051483128514031005180314D30D19
:1000E0008510D40B6B288316051083125308080063
:1000F0000510851485100514080005148514851055
:10010000080083018B0185010730990083163C307C
:10011000850034309700950070308F0008308100E2
:10012000831281018B128B17051485145B221E200C
:100130000C3008200230CB00803008200030CF0087
:10014000BD30D0003820C030082038206C226C220E
:10015000803008203820C030082038206C226C22E3
:10016000CB0B9C28013008206C226C22EA206F21E6
:10017000C60146150630C500152946346D34533482
:1001800074346534723465346F3400342034203470
:1001900052346134643469346F342034003456345A
:1001A00065347234203431342E34303434340034F5
:1001B00020346234793420344D342E345934203490
:1001C0000034203456346F346C343D3420342034C1
:1001D00020340034831626309B0083124330840081
:1001E0000230CB0083161C141A089B0A831280006D
:1001F000840ACB0BF2280800831626309B0083125A
:10020000433084000230CB00000883169A001C158E
:1002100055309D00AA309D009C149C180D299B0A06
:100220008312840ACB0B04290800851E3B21051E7E
:100230004821851D5521051D6121461C2C296F2152
:10024000461057228B120530C2003830810027300B
:10025000C0001030C1008B16461D36294908CF005A
:100260004A08D0004611C03008203820C61C152985
:10027000FC20C61015295722851A45294614C303A8
:10028000430A031D45294508C300851E452908006A
:100290005722051A52294614C30A43084502031877
:1002A0005229C301051E52290800572285195E29CB
:1002B0004614C403440A031D5E29C401851D5E293A
:1002C0000800572205196C294614C40A44080F3C3B
:1002D00003186C290F30C400051D6C29080001307B
:1002E000CF00AF30D0004308C9000310C90DC90DBD
:1002F0004908CA00C90D490D0318CF0A4A07031857
:10030000CF0AD0070318CF0A8030082038204F08C2
:10031000C9005008CA000930D0070318CF0A44208A
:10032000C700D00A0319CF0A4420C800C0300820F3
:100330000030CF00E130D00038200A3044020318EA
:10034000A529C63008204408AB29C5300820313023
:100350000B200A30440230380B203B220800433483
:100360004F342E3443344F342E344C344F34003415
:100370002034373436342E3435344D3448347A34DE
:1003800000340134583442346534483461347034B4
:1003900070347934213400342034373438342E34F6
:1003A00039344D3448347A340034073458344634C0
:1003B0004D3420344F34533441344B3441340034C1
:1003C0002034383435342E3431344D3448347A3492
:1003D00000341634D8344E3448344B342034463448
:1003E0004D342034203400342034383438342E3422
:1003F00031344D3448347A3400341E3458344D345A
:100400004234533420342034203420342034003417
:100410002034393430342E3436344D3448347A3440
:100420000034243498344F3442344334203420345C
:1004300020342034203400342034393431342E3404
:1004400039344D3448347A3400342734D834413484
:1004500042344334203420342034203420340034D7
:100460002034393433342E3433344D3448347A34F0
:1004700000342B345834482020305120D0305120C3
:1004800001305120470851204808512000305120A8
:1004900000305120883051204408803851204D20B0
:1004A00008002730CC00542ACC0B532A08001E30F9
:1004B0005E2A64305E2AC8305E2A0130CD00DD300D
:1004C000CC00622A632A642ACC0B612A0000682AC5
:1004D000692ACD0B5F2A08000A30CE005922CE0BC4
:1004E0006E2A0800F0000308F10083120B1D922A07
:1004F0000B11383081000130C1020319832A03181F
:10050000922AC002922AC008031D922A2730C000F6
:100510001030C1000530420203194615C20B922A61
:0E052000C6148B1271088300F00E700E0900D5
:02400E00C43FAD
:1042000043006F0070007900720069006700680069
:1042100074002000280043002900200032003000F4
:10422000320030002D00320030003200310020001A
:104230006200790020004D002E00590061006D00E1
:1042400061006D006F0074006F00FF00030001004B
:00000001FF
